:10000E00323032322D30372D3132202D20313233F5
:05001E00343536370007
:102692007BFF7A00790E7D2D123807EA494B601FC5
:1026A2007BFF7A00790E7D2D123807E92402F9E4C6
:1026B2003AFA90046CEBF0A3EAF0A3E9F08004E4A8
:1026C200FEFF2290046CE0FBA3E0FAA3E0F9900085
:1026D20001121E01FFC39430400CEFD3943950060F
:1026E200EF24D0FF801A900001121E01FFC39461F3
:1026F200400CEFD394665006EF24A9FF80027F00BE
:10270200EF7D00FC121DE8FFC39430400CEFD39420
:10271200395006EF24D0FF802290046CE0FBA3E046
:10272200FAA3E0F9121DE8FFC39461400CEFD394C1
:10273200665006EF24A9FF80027F00EFC454F04CDC
:10274200FC90046CE0FBA3E0FAA3E0F99000021213
:102752001E01FFC39430400CEFD394395006EF248E
:10276200D0FF801A900002121E01FFC39461400C38
:10277200EFD394665006EF24A9FF80027F00EF7525
:10278200F010A4FFE5F04CFEEF4DFF900003121E87
:1027920001FDC39430400CEDD394395006ED24D0A2
:1027A200FD802590046CE0FBA3E0FAA3E0F9900021
:1027B20003121E01FDC39461400CEDD394665006D2
:0B27C200ED24A9FD80027D00EF4DFF1B
:0127CD0022E9
:1020E300E47880F612422FC290E4F5A775E101F57A
:1020F300E275E34043C91090046AF0A3F090046BC7
:10210300E004F0700690046AE004F090046AE07062
:1021130004A3E0640E70E643B28FE4F5A91241A074
:10212300E4FF1240E443EF04E490046AF0A3F09068
:10213300046AE0FEA3E0FFC39402EE940050157D11
:1021430001123F9A90046BE004F070E390046AE09C
:1021530004F080DBE4F520C20AC208C20EC20DC23D
:102163000CD20F7880F608F67826F618F6782CF657
:1021730090046AF0A3F090046AE0FEA3E0FFC3EECC
:102183009401501C744D2FF58274023EF583E4F0E4
:1021930090046BE004F070DE90046AE004F080D6F3
:1021A300E490046AF0A3F090046AE0FEA3E0FFC3A6
:1021B3009440EE9400501C744D2FF58274033EF549
:1021C30083E4F090046BE004F070DC90046AE004B4
:1021D300F080D4124291E4F5A7E5EF20E10CE5EF9E
:1021E3005408D394004003D38001C392037D08E4D1
:1021F300FF124076E4782BF67823F690024AE0FB50
:10220300A3E0FAA3E0F97823E6FF75F010A4F582C2
:1022130085F083121E01FE782B26F6EE60057823E7
:102223000680D8EFD39400403590024AE0FBA3E048
:10223300FAA3E0F990000D121F9E121DE8FF7455DA
:10224300121E2E121DE864556002D20C74AA121ECF
:102253002E121DE864AA6002D20CEF121E2EE5EFC7
:102263005402D3940040047F018002E4FF122554FA
:10227300900469EFF0900469E020E03CC20974FF28
:10228300782EF608F608F608F67E007F107D007BB0
:10229300007A00793412202590046F74FFF0A37440
:1022A3000AF0A374A7F0A3E4F0A37410F07B007A00
:1022B3000079341239DD8002D2091226927832A6CF
:1022C3000608A607900469E030E1030223A6E4A30D
:1022D300F0A3F090046BE0C4F8540FC868FF9004B7
:1022E3006AE0C454F048FE90024AE0FBA3E0FAA37C
:1022F300E0F98F828E83121E01700302239DE92F62
:10230300F9EA3EFA900004121E0120E27CE49004F4
:1023130068F0900468E0FDC3781E96506C90046BDF
:10232300E0C4F8540FC868FF90046AE0C454F0484E
:10233300FE90024AE0FBA3E0FAA3E0F98F828E83CA
:10234300121E01FF7E00C006C0077C0090046BE0F4
:10235300C4F8540FC868FF90046AE0C454F048FE00
:10236300E92FF9EA3EFA90000D121F9E782BE68DB5
:10237300F0A429F9EA35F0FA7D00D007D00612203F
:1023830025900468E004F0808990046BE004F07009
:102393000690046AE004F00222D67F011227CEC21F
:1023A3000B8007E4FF1227CED20BE490046AF0A35C
:1023B300F090046AE0FEA3E0FFC39402EE940050A1
:1023C300197A007B967D0312370290046BE004F0C8
:0A23D30070DF90046AE004F080D788
:0123DD0022DD
:05428C00782CE6FF2282
:06427400EF24FF920F226F
:06427A00A20FE433FF2255
:03002300022A208E
:102A2000C0E0C0F0C083C082C0D075D000C000C07C
:102A300001C002C003C004C005C006C007309944ED
:102A4000C2997826067926E77881667018F6782686
:012A5000F68F
:102A5100900452740AF000900452E014F0E070F611
:042A6100C290801F80
:102A65009004527414F000900452E014F0E070F6F3
:102A75007826E6244DF582E43403F583E0F59920C4
:102A85009803022B28209A08200A05C298022B24B5
:102A9500C29A7825E606244DF582E43402F583E5ED
:102AA50099F0C298E6FFB4011290024DE0FE700362
:102AB500F68070EE54072402782DF6EFB4020D78F7
:102AC5002DE6B4090790024EE02403F67825E6FFCB
:102AD500FD7C00B40007ECB40103F68046EFC37833
:102AE5002D96403FED24FFFDEC34FFFC7B017A027F
:102AF500794D12314A7825E6244CF582E43402F505
:092B050083E06F60047600801A81
:102B0E009004527414F000900452E014F0E070F649
:102B1E00782A0612002678257600D007D006D00532
:102B2E00D004D003D002D001D000D0D0D082D08338
:052B3E00D0F0D0E032F0
:05429100782AE6FF227F
:1031FA0090024EE075F010A4FF90024AE0FBA3E0B3
:10320A00FAA3E02FF9EA35F0FA90000D121F9E900A
:10321A000455782CE6FF18E68FF0A4FFE02FF5821C
:0F322A00E435F0F583121E01FF7B017A0479531E
:10323900900462EFF0A3EBF0A3EAF0A3E9F09004A5
:1032490063E0FBA3E0FAA3E0F9EA494B60229004AA
:1032590063A3A3121DE8FF900462E0FD7C00124203
:1032690020900463E0FBA3E0FAA3E0F9EF121E2E1D
:103279009004667414F000900466E014F0E070F6AF
:10328900900462E0F5997F01123EFF3099FDC299E1
:013299002212
:103AA80090034D7478F07825E6244CF582E43402CE
:093AB800F583E090034EF07F025B
:103AC10090FFFF121FF4EFF090FFFF121FF4850823
:0B3AD10083850982A3E07881F6D29083
:103ADC008508838509827414F0850883850982E042
:0B3AEC00D39400400600E014F080EED0
:0C3AF70090034DE0F599900002021FF4CE
:103B0300C9EFC9E964017028EDC39B403E781EE606
:103B1300FFEB2FFFE433FEEDC39FEE6480F8748068
:103B2300985028D20AC3ED9B782CF6782776012289
:103B3300CFE9CFEFB4021ACFEBCFCEEDCEEE6F705D
:103B43000AD20A782CF67827760222C20AE478276A
:023B5300F62258
:10356C00900462ECF0A3EDF0C9EFC9BAFF19BBFFF0
:10357C0016900462E06A7003A3E06B7067D20A785D
:10358C002CF67827E9F622E964017035C3900463C0
:10359C00E09B900462E09A4026781EE62BFFE43A0A
:1035AC00FEE0FCA3E0FDC39FEC9E5013D20ACFEBD0
:1035BC00CFCEEDCEC3EE9F782CF678277601228005
:1035CC0023CFE9CFEFB40222CEEACECFEBCF9004DB
:1035DC0062E06E7003A3E06F700AD20A782CF67862
:0B35EC0027760222C20AE47827F622AC
:1000260090024DE0FE54F8900454F0EE121FCE00FC
:100036007209007F0A009210009B1100AC1200C3E7
:100046001900D91A00FE2001042801982902D93383
:10005600031437035039036A41037549038050037B
:10006600D46102A37003CC980000040490024EE011
:10007600FD782FE6FB7F01802790024EE0FCA3E08F
:10008600FD782EE6FA08E6FB7F01802BD20A782758
:10009600760302040490024EE0FD7831E6FB7F020F
:1000A600123B0302040490024EE0FCA3E0FD78300C
:1000B600E6FA08E6FB7F0212356C02040490024E53
:1000C600E0FD782FE6FB7F01123B03200A030204C2
:1000D60004801A90024EE0FCA3E0FD782EE6FA08B2
:1000E600E6FB7F0112356C200A0302040490034DDF
:1000F6007478F07F0102040175EF10020404C2ACAB
:10010600E4900453F0D2907B017A0479537F7F12F6
:1001160032397B017A0479537F181232397B017A9E
:100126000479537F051232397823E6123232782E5B
:10013600E6123232782FE61232327830E612323256
:100146007831E61232327832E61232327833E612FB
:100156003232E4900455F0900455E0FFC3941050F9
:100166001074342FF8E6123232900455E004F08011
:0F017600E6900453E0FF7B007A007900123239E3
:10018500900461740AF000900461E014F0E070F6E8
:1001950002028E90024EE0FFC378239640030202CE
:1001A50095EF75F010A4FF90024AE0FBA3E0FAA3D7
:1001B500E02FF9EA35F0FA90045EEBF0A3EAF0A33C
:1001C500E9F0C2ACE4900453F0D2907B017A047953
:1001D500537F7F1232397B017A0479537F0D1232B6
:1001E5003990045EE0FBA3E0FAA3E0F9121DE812E2
:1001F500323290045EE0FBA3E0FAA3E0F99000013F
:1002050012322F90045EE0FBA3E0FAA3E0F9900020
:100215000212322F90045EE0FBA3E0FAA3E0F9900E
:10022500000312322F90045EE0FBA3E0FAA3E0F98D
:1002350090000412322FE4900455F0900455E0FF2D
:10024500C39408502690045EE0FBA3E0FAA3E024E3
:1002550005F9E43AFA7E00E92FF9EE3AFA121DE8BB
:10026500123232900455E004F080D0900453E0FF40
:090275007B007A00790012323995
:10027E00900461740AF000900461E014F0E070F6EE
:10028E00C290D2AC02040490034D7478F0E4A3F053
:10029E007F020204011242567844121F3C90034D15
:1002AE00747CF07844E6A3F008E6A3F008E6A3F029
:1002BE0008E6A3F07C007D057B017A03794D1231AF
:1002CE004A900352EFF07F0602040190024EE0FFC7
:1002DE00B4010FA3E0FDA3E0782ECDF608EDF602F3
:1002EE0003CCEFB4020A90024FE0782EF60203CC54
:1002FE0090024EE0B4030CA3E0FFA3E07830CFF6FB
:10030E0008EFF60203CCE4900455F0900455E0FF9C
:10031E00C39410502790024EE0FEEFC39E501D90E6
:10032E000455E0244FF582E43402F583E0FE743484
:10033E002FF8EEF6900455E004F080CFE47843F603
:10034E00807C7A007B327D01782CE6FF123702909A
:10035E00024EE0FDE4FF12407602040490024EE0ED
:10036E0024FF920202040490024EE024FF92010246
:10037E000404782CE660089004577402F0800E9006
:10038E000457200D057403F080037401F090034DA3
:10039E007479F0900457E090034EF07C007D027B60
:1003AE00017A03794D12314A90034FEFF07F031219
:1003BE003AC1900457E06401703CD20E8002D2081C
:1003CE00788076F180307A007B327D017F001237A3
:1003DE000290034D7479F090024EE090034EF07C43
:1003EE00007D027B017A03794D12314A90034FEF63
:1003FE00F07F03123AC1900454E064A06003020639
:10040E009B781EE6B4010E300F0B7A007B327D0115
:10041E007F0112370290024DE064A1600302054E87
:10042E00A3E0C3782396400302054390024AE0FB03
:10043E00A3E0FAA3E0F990024EE0FF75F010A4F5E8
:10044E008285F083121E01900457F0EF75F010A410
:10045E00FFE92FF9EA35F0FA900004121E0130E29E
:10046E003C90024EE0FF120003900457EFF0900311
:10047E004D747FF0A3EFF02402FDE433FC7B017A90
:10048E0003794D12314A900457E0FE244FF582E471
:10049E003403F583EFF0EE2403FF02069890024E2C
:1004AE00E0FF120003C2ACE4900453F0D29090042B
:1004BE0057E0D3940640377B017A0479537F7F123D
:1004CE003239900457E0123232E4900455F0900421
:1004DE0057E0FF900455E0C39F500B1231FA900481
:1004EE0055E004F080E8900457E004F08026900474
:1004FE0057E02478123232E4900455F0900457E01D
:10050E00FF900455E0C39F500B1231FA900455E052
:10051E0004F080E8900453E0FF7B007A007900122B
:02052E00323960
:10053000900461740AF000900461E014F0E070F639
:1005400002068A90034D7478F07F010206989002AB
:100550004DE064A2600302069B7823E6FFA3E0FE61
:10056000C39F4003020690A3E0FDC39F4003020621
:1005700090EE9D400302069090024EE0900455F0EC
:10058000E490045CF0A3F090024FE0FE900455E08C
:10059000FFD39E503412000390024AE0FBA3E0FA1E
:1005A000A3E0F9900455E075F010A4F58285F0837E
:1005B000121E01FF90045DE02FF090045CE0340017
:1005C000F0900455E004F080BEC2ACE4900453F017
:1005D000D2907B017A0479537F7F12323990045C88
:1005E000E0FEA3E0FFC39480EE94005002800F90E1
:1005F000045CE0448012323290045CA3E0FF1232CB
:100600003390024EE0900455F090024FE0FF9004CA
:1006100055E0D39F5056E4A3F090024AE0FBA3E0DC
:10062000FAA3E0F9900455E0FF75F010A4F5828577
:10063000F083121E01FE900456E0C39E5026EF7513
:10064000F010A4FF90024AA3A3E02FF9EA35F0FAD4
:1006500090000D121F9E90045612321C900456E01A
:1006600004F080B5900455E004F0809D900453E0C0
:0A067000FF7B007A00790012323996
:10067A00900461740AF000900461E014F0E070F6EE
:10068A00C290D2AC800B90034D7478F07F01123A7D
:10069A00C1900454E064587057FA7B327D01782C7B
:1006AA00E6FF1237029004657401F0A37403F0A305
:1006BA00744EF07B017A02794E123C4A900457EF4D
:1006CA00F0E0FE247890034DF0EE2401FDE433FCC3
:1006DA007B017A03794D12314A900457E0FE244E89
:1006EA00F582E43403F583EFF0EE2402FF123AC1F7
:1006FA00900454E0FF64806008EF64886003020994
:10070A0003300F367827E6B4010F7A007B327D0179
:10071A00782CE6FF1237028021E4900455F0900409
:10072A0055E0FFC3781E9650117A007B327D011284
:10073A003702900455E004F080E490024DE054073B
:10074A00FF900457F0BF07139004567401F090020B
:10075A004EE0900457F090024F8008E4900456F05F
:10076A0090024EE0900458F0900457E014F0A3E091
:10077A00FFC3782396400302090390024AE0FBA3D1
:10078A00E0FAA3E0F975F010EFA4F58285F0831280
:10079A001E01FF900457E0D39F4002EFF07827E64E
:1007AA00B4010D782CE690045BF090045AF0800BAB
:1007BA00E490045AF0781EE614A3F090045AE07804
:1007CA002CF690045BE0FF782CE6D39F40030208E6
:1007DA00F2E4900455F0900457E0FF900455E0C30A
:1007EA009F40030208E4900458E075F010A4FF90BB
:1007FA00024AE0FBA3E0FAA3E02FF9EA35F0FA9007
:10080A000004121E0130E2030208DB900001121EEE
:10081A00016438704F900457E0D39404900455E073
:10082A00FF4010A3E02F244FF582E43402F583E061
:10083A00FD807E7825E6C39FFFE49400FE744B2F6B
:10084A00F58274023EF583E0FD900458E075F010DD
:10085A00A4FF90024AE0FBA3E0FAA3E02FF9EA35ED
:10086A00F0FA804D90024AE0FBA3E0FAA3E0F99087
:10087A000458E075F010A4F58285F083121E01FF7A
:10088A007825E6C39FFFE49400FE900455E07C00BF
:10089A002FFFEC3EFE744C2FF58274023EF583E086
:1008AA00FD900458E075F010A4FFE92FF9EA35F03D
:1008BA00FA90000D121F9E782CE6FF18E68FF0A41E
:1008CA00FF900455E02FF582E435F0F583ED121E12
:1008DA0040900455E004F00207E0900458E0FF124B
:1008EA004105782C060207CC90045AE0782CF69041
:1008FA000454E0B48803123AA8900454E064A8604F
:10090A0003020AA6300F367827E6B4010F7A007B75
:10091A00327D01782CE6FF1237028021E4900455DB
:10092A00F0900455E0FFC3781E9650117A007B328E
:10093A007D01123702900455E004F080E490024EE3
:10094A00E030E718547FFEA3E0FDEDFF90045CEE73
:10095A00F0A3EFF09004567403F0801390024EE077
:10096A00FF90045CE4F0A3EFF09004567402F09058
:10097A000456E0FF244DF582E43402F583E0FE7468
:10098A004E2FF582E43402F583E0900459F0CFEE5D
:10099A00CF900458EFF0900459E0FF900458E0FE1D
:1009AA00D39F4003020AA3EEC37823964003020AA8
:1009BA009A90024AE0FBA3E0FAA3E0F975F010EE80
:1009CA00A4F58285F083121E01900457F07827E679
:1009DA00B4010D782CE690045BF090045AF0800B79
:1009EA00E490045AF0781EE614A3F090045AE078D2
:1009FA002CF690045BE0FF782CE6D39F4003020AB2
:100A0A0088E4900455F0900457E0FF900455E0C341
:100A1A009F505D900458E075F010A4FF90024AE0E0
:100A2A00FBA3E0FAA3E02FF9EA35F0FA90000412EA
:100A3A001E0120E233900455E0FFA3E02F244FF576
:100A4A0082E43402F583E0FD90000D121F9E782C9B
:100A5A00E6FF18E68FF0A4FF900455E02FF582E434
:100A6A0035F0F583ED121E40900455E004F08096AF
:100A7A00900458E0FF124105782C060209FC900404
:100A8A005AE0782CF6900457E0FF900456E02FF0D5
:0C0A9A00900458E004F00209A0123AA8F1
:010AA600222D
:10F000007880E664F1600302F6B3784EF608F6788D
:04F0100081E6602114
:10F01400900468740AF000900468E014F0E070F65C
:10F02400784F06E618700106784EB627DE08B6104B
:10F03400DAC2AFE4784AF618F6209833E4784EF64C
:10F0440008F6209826C3784FE6948818E69413505F
:01F054001AA1
:10F05500900468740AF000900468E014F0E070F61B
:10F06500784F06E61870DA0680D7B29780CA7849D5
:10F07500A699C298E6FF641A6008EF640A60030265
:10F08500F16DE4784EF608F6209826C3784FE6949D
:07F095008818E69413501ADD
:10F09C00900468740AF000900468E014F0E070F6D4
:10F0AC00784F06E61870DA0680D7309884784AA62E
:10F0BC0099C298E4784EF608F6209826C3784FE665
:08F0CC00948818E69413501A11
:10F0D400900468740AF000900468E014F0E070F69C
:10F0E400784F06E61870DA0680D720980302F03DC0
:10F0F400784AA699C298E4784EF608F6209826C372
:0BF10400784FE6948818E69413501A28
:10F10F00900468740AF000900468E014F0E070F660
:10F11F00784F06E61870DA0680D720980302F03D84
:10F12F00784AA699C29818E6641A600302F6A4D228
:03F13F0090C299E2
:10F142009004687414F000900468E014F0E070F623
:06F152007599783099FD6B
:10F15800900468740AF000900468E014F0E070F617
:10F16800C29002F6A47849E6FF6450600302F211E7
:10F17800784EF608F6209826C3784FE6948818E665
:04F188009413501A72
:10F18C00900468740AF000900468E014F0E070F6E3
:10F19C00784F06E61870DA0680D720980302F03D07
:0AF1AC00784AA699C298D290C29941
:10F1B6009004687414F000900468E014F0E070F6AF
:08F1C6007599793099FDC29999
:10F1CE009004687414F000900468E014F0E070F697
:08F1DE007599013099FDC299F9
:10F1E6009004687414F000900468E014F0E070F67F
:06F1F600E4F5993099FDDB
:10F1FC00900468740AF000900468E014F0E070F673
:0EF20C00C29002F6A4EF64017047D290C2993E
:10F21A009004687414F000900468E014F0E070F64A
:08F22A007599783099FDC29935
:10F232009004687414F000900468E014F0E070F632
:06F24200E4F5993099FD8E
:10F24800900468740AF000900468E014F0E070F626
:10F25800C29002F6A47849E66402600302F33578A6
:10F268004EF608F6209826C3784FE6948818E69458
:03F2780013501A16
:10F27B00900468740AF000900468E014F0E070F6F3
:10F28B00784F06E61870DA0680D720980302F03D17
:10F29B00784AA699C298E408F618E6FF13B392973A
:10F2AB00EF25E0FECC74F0CCCD7400CDC3E49DEE25
:10F2BB009C502AE67F0025E0FEC39460501FE4F5C6
:10F2CB00A7758F037850EEF608EFF675B7A5788023
:10F2DB00E6F5B78F828E83E4F0F58F8004784B765A
:05F2EB00FFD290C29962
:10F2F0009004687414F000900468E014F0E070F674
:08F300007599783099FDC2995E
:10F308009004687414F000900468E014F0E070F65B
:08F31800784BE6F5993099FDF0
:10F32000900468740AF000900468E014F0E070F64D
:10F33000C29002F6A47849E66403600302F494786C
:10F340004EF608F6209826C3784FE6948818E6947F
:03F3500013501A3D
:10F35300900468740AF000900468E014F0E070F61A
:10F36300784F06E61870DA0680D720980302F03D3E
:10F37300784AA699C298E4784EF608F6209826C3F0
:0BF38300784FE6948818E69413501AA7
:10F38E00900468740AF000900468E014F0E070F6DF
:10F39E00784F06E61870DA0680D720980302F03D03
:10F3AE00784CA699C298784AE6FF139297EF25E01B
:10F3BE00FECC74F0CCCD7400CDC3E49DEE9C400326
:10F3CE0002F03DE67D0025E0FCC39460400302F0B0
:10F3DE003DE4F5A7758F01784CE675F020A42DFF5E
:10F3EE00E5F03C7850F608EFF6E4784DF6784DE609
:10F3FE00C394205047E408F608F6209816C3784FB9
:10F40E00E6948818E69413500A000806E61870EA87
:10F41E000680E720980302F03D75B7A57880E6F5E3
:10F42E00B778500806E618CEE6CE70010614F582BF
:10F43E008E83E599F0C298784D0680B1E4F58FD2AF
:03F44E0090C299D0
:10F451009004687414F000900468E014F0E070F611
:08F461007599783099FDC299FC
:10F469009004687414F000900468E014F0E070F6F9
:06F47900E4F5993099FD55
:10F47F00900468740AF000900468E014F0E070F6ED
:10F48F00C29002F6A47849E6FD6404600302F55DBC
:10F49F00784EF608F6209826C3784FE6948818E63B
:04F4AF009413501A48
:10F4B300900468740AF000900468E014F0E070F6B9
:10F4C300784F06E61870DA0680D720980302F03DDD
:10F4D300784AA699C298E625E07852F608E4F678C9
:10F4E3004BF6784EF608F678520806E618CEE6CEC6
:10F4F30070010614F5828E83E493784B26F6784FD9
:10F5030006E618700106784FE6700418E664027088
:05F51300D6D290C29960
:10F518009004687414F000900468E014F0E070F649
:08F528007599783099FDC29934
:10F530009004687414F000900468E014F0E070F631
:08F54000784BE6F5993099FDC6
:10F54800900468740AF000900468E014F0E070F623
:10F55800C29002F6A4ED6405600302F69B784EF6AD
:10F5680008F6209826C3784FE6948818E694135036
:01F578001A78
:10F57900900468740AF000900468E014F0E070F6F2
:10F58900784F06E61870DA0680D720980302F03D16
:10F59900784AA699C298E4784EF608F6209826C3C8
:0BF5A900784FE6948818E69413501A7F
:10F5B400900468740AF000900468E014F0E070F6B7
:10F5C400784F06E61870DA0680D720980302F03DDB
:0AF5D400784CA699C298D290C29913
:10F5DE009004687414F000900468E014F0E070F683
:08F5EE0075997F3099FDC29967
:10F5F6009004687414F000900468E014F0E070F66B
:10F606007599203099FD784AE625E0FC784CE67538
:10F61600F020A42400FFE5F03C7852F608EFF6E46B
:08F62600784BF6784DF6C2990D
:10F62E009004687414F000900468E014F0E070F632
:10F63E007852E6FE08E6F5828E83E493F5993099CA
:10F64E00FD78520806E618CEE6CE70010614F58255
:10F65E008E83E493784B26F6784D06E6B420BFC22F
:01F66E009902
:10F66F009004687414F000900468E014F0E070F6F1
:08F67F00784BE6F5993099FD86
:10F68700900468740AF000900468E014F0E070F6E3
:10F69700C29080097849E6B4060375EF107849E609
:0CF6A7006407600302F03D7880F6D2AFEB
:01F6B3002234
:10396F007F00123EFF20090B7A007B327D017F0022
:10397F00123702300C0B7A007B1E7D017F0012374D
:10398F0002300817300D147A007B327D01782CE657
:10399F00FF123702C208122E1CD209200B0C300D59
:1039AF0009788076F1122E1CD20B300E0B300D08D9
:1039BF00C20E12422F12F000200D1212424CE47B65
:0E39CF002C7A01F9F8C3121F1F5002D20D22EC
:1041640075EF027F64DFFE1220E312428C1241F4E9
:0E417400E4FFFE123D2C12396F1212CC80F8BF
:102B4300005EBCE2613FDD83C29C7E20A3FD1F418A
:102B53009DC3217FFCA2401E5F01E3BD3E6082DC7A
:102B6300237D9FC1421CFEA0E1BF5D0380DE3C626A
:102B7300BEE0025CDF81633D7C22C09E1D43A1FF5A
:102B83004618FAA427799BC584DA3866E5BB59074A
:102B9300DB856739BAE406581947A5FB7826C49A3A
:102BA300653BD987045AB8E6A7F91B45C6987A242A
:102BB300F8A6441A99C7257B3A6486D85B05E7B91A
:102BC3008CD2306EEDB3510F4E10F2AC2F7193CD0A
:102BD300114FADF3702ECC92D38D6F31B2EC0E50FA
:102BE300AFF1134DCE90722C6D33D18F0C52B0EEEA
:102BF300326C8ED0530DEFB1F0AE4C1291CF2D73DA
:102C0300CA947628ABF517490856B4EA6937D58BC9
:102C13005709EBB536688AD495CB2977F4AA4816B9
:102C2300E9B7550B88D6346A2B7597C94A14F6A8A9
:102C3300742AC896154BA9F7B6E80A54D7896B3599
:0A2C43000000000000002B96B9DD30
:033C9A0001130A09
:1041F400900468121F6DFFFFFFFF900468E0FCA3AA
:08420400E0FDA3E0FEA3E0FFD2
:01420C00228F
:10314A0090FFFE121FF4ECF0A3EDF090FFFD121FAA
:0F315A00F4EBF0A3EAF0A3E9F090FFFC121FF4EE
:10316900850883850982A3A3E4F0850883850982FC
:10317900F0A3F0900007122018E0FEA3E0FF8508F5
:1031890083850982E0FCA3E0FDC39FEE6480F8EC2F
:10319900648098504C900004122018E0FBA3E0FAD8
:1031A900A3E0F98D828C83121E01FF8508838509AE
:1031B90082A3A3E06FFF900003122018EFF09000A4
:1031C90003122018E0902B4393850883850982A375
:1031D900A3F0850883850982E475F001121E9880A1
:0B31E90092850883850982A3A3E0FF04
:0631F400900009021FF427
:0E422000CEEDCEEE6F7848F6E6902B4393FF7E
:01422E00226D
:10407600EF7020F5A77598D0E589540F4420F5898F
:10408600438E08CFEDCFEF902C4293F58DD28ED292
:05409600ACC2BCD2AF7A
:01409B002202
:103BF9007816121F5400000000781A121F54000092
:103C09000000780A7664E47849F67849E6FFC394B7
:103C190002502DEF25E025E0240BF8E4F6EF25E02E
:103C290025E0240CF8E4F6EF25E025E0240DF8E47E
:103C3900F6EF25E025E0240EF8E4F678490680CA77
:013C49002258
:1041A000D2AFD2A9C2BBE589540F4401F589758EFF
:0C41B00002758CECE4F58AD28C023BF91D
:062FD20090FFFF121FF446
:102FD800850883850982E4F0850883850982E0FFF6
:102FE800C39402400302308BEF25E025E0240EF85D
:102FF800E6FFD39400406EE025E025E0240CF8E6D7
:103008007063EF30E013E0FF25E025E0240EF8E6DA
:10301800D3940140047D00800A7D018508838509D9
:1030280082E0FF123A45850883850982E0FF25E0A2
:1030380025E0240EF8E6B401057D01123A4585081D
:1030480083850982E0FF25E025E0240EF816E66076
:1030580014EF25E025E0240DF8E6FEEF25E025E055
:10306800240CF8EEF6850883850982E025E025E042
:10307800240CF8E6600116850883850982E004F0CF
:03308800022FE034
:06308B00900001021FF499
:03000B000235F7C4
:1035F700C0E0C0F0C083C082C0D0E8C0E0E9C0E04E
:10360700EAC0E0EBC0E0ECC0E0EDC0E0EEC0E0EF08
:10361700C0E0758CEC7816121F30EF2401FFE43EF2
:10362700FEE43DFDE43CFC7816121F3C780A16E6E2
:10363700701B781A121F30EF2401FFE43EFEE43DB1
:10364700FDE43CFC781A121F3C780A7664122FD2EC
:103657001240C2D0E0FFD0E0FED0E0FDD0E0FCD0C9
:10366700E0FBD0E0FAD0E0F9D0E0F8D0D0D082D0BB
:0636770083D0F0D0E03228
:103F9A0090FFFF121FF4EDF090FFFF121FF4EFF0F5
:103FAA00850883850982E0FFC39402500DA3E0FED1
:103FBA00EF25E025E0240BF8EEF6900002021FF44C
:1037020090FFFE121FF4EAF0A3EBF090FFFF121FEE
:10371200F4EDF090FFFF121FF4EFF08508838509A6
:1037220082E0FFC394025056EF25E025E0240EF814
:10373200E6704BE0FB25E025E0240CF8E6703FA3A1
:10374200E025E004FF850883850982E0FA25E0256B
:10375200E0240EF8EFF6850883850982A3A3E0FE34
:10376200A3E0FF7C007D0A121E62EA25E025E02428
:103772000DF8EFF6EB25E025E0240CF8E4F69000D6
:0437820004021FF42A
:103A450090FFFF121FF4EDF090FFFF121FF4EFF04F
:103A5500850883850982E0FFC39402501EEF25E0A7
:103A650025E0240BF8E66013A3E070047F018002D3
:103A75007F00850883850982A3EFF0850883850982
:103A850082E0FF7008A3E024FF92978010EFB40155
:103A95000C850883850982A3E024FF92A09000028B
:033AA500021FF409
:09424C00C2AF7816121F30D2AF88
:014255002246
:09425600C2AF781A121F30D2AF7A
:01425F00223C
:103EFF0090FFFF121FF4EFF0850883850982E070B1
:103F0F00057814F608F63010167813E675F064A4E9
:103F1F00FFC37815E69F18E695F05003E4F5D390AC
:053F2F000001021FF477
:1040E400D210E47814F608F6EF78136003F6800231
:1040F400760AE4F5D975D2FF75D940F5D375EF0684
:014104002298
:0F422F00C210E47814F608F6781376FFF5D9225A
:1040C200781506E6187001063010167813E675F0BA
:1040D20064A4FFC37815E69F18E695F05003E4F553
:0240E200D322E7
:083D2C0090046FEEF0A3EFF02C
:103D3400E4A3F0A3F090046FE0FEA3E0FFC39004BB
:103D440072E09F900471E09E501C7FE87E0312385D
:103D5400817F01123EFF900472E004F070D790045A
:063D640071E004F080CFC5
:013D6A002236
:0838810090047CEEF0A3EFF0CF
:10388900D394FAEE9400501990047CA3E0FFEFD38F
:103899009400405C000000000000000000001F8050
:1038A900ED90047CE0FFA3E090047FCFF0A3EFF05C
:1038B900D3900480E094FA90047FE0940040177F4D
:1038C900FA7E00123881900480E02406F090047F8B
:1038D900E034FFF080DAD390047DE0940090047C1A
:1038E900E09400400B90047FE0FEA3E0FF123881D2
:0138F90022AC
:10329A009004787401F0A37404F0A37472F07B01B3
:0632AA007A0479707D0238
:0E32B000900474EBF0A3EAF0A3E9F0A3EDF0B4
:1032BE007F01123EFF900478E0FBA3E0FAA3E0F951
:1032CE00121EAE2400FFE5F03460FE900474E0F9A7
:1032DE00A3E0FAA3E090047BC9F0A3EAF0A3E9F01F
:1032EE00E4FD900477E0FCEDC39C5022EF2DF582B7
:1032FE00E43EF583E493FC90047BE0FBA3E0FAA3A9
:10330E00E0F98D82758300EC121E400D80D490047E
:10331E0077E0FFA3E0FBA3E0FAA3E0F9E48FF0026D
:02332E001ED9A6
:102D3D0090046A7412F0A37434F09004727401F06C
:102D4D00A37404F0A3746CF07B017A04796A7D029C
:0E2D5D0090046EEBF0A3EAF0A3E9F0A3EDF012
:102D6B007880E664F16003022E1B12422FC2AFE49F
:102D7B00F5A7758F01A3E0FBA3E0FAA3E0F9121E00
:102D8B00AE2400FFE5F034607849F608EFF69004C6
:102D9B006EE0FBA3E0FAA3E0F9784DC6EBC608C6DC
:102DAB00EAC608C6E9C6E4784BF6900471E0FF78F2
:102DBB004BE6C39F503C784DCBE6CB080806E61894
:102DCB00CAE6CA70010614F9121DE8784CF675B7FD
:102DDB00A57880E6F5B7784CE6FF78490806E61843
:102DEB00CCE6CC70010614F5828C83EFF0784B06A1
:102DFB0080B8E4F58F900471E0FFA3E0FBA3E0FA49
:102E0B00A3E0F9E48FF0121ED9D2AFE4FF1240E435
:012E1B002294
:103CE6007880E664F1703EC2AF12422FE4F5A77504
:103CF6008F03784A766008F67849F675B7A5788016
:103D0600E6F5B7784AE6FE08E6F5828E83E4F02605
:103D1600F618740236F61806E6B408DFE4F58FD214
:053D2600AFFF1240E4B4
:013D2B002275
:102E1C00123CE6E490046CF0A3F07B019004720485
:102E2C00F0A37404F0A3746CF01B7A00792E7D1659
:102E3C00122D5D122D3DE4900469F0900469E0C3FD
:102E4C00781E964003022EF1E4900468F090024A3A
:102E5C00E0FBA3E0FAA3E0F9900468E0FF75F01042
:102E6C00A4F58285F083121E016071EF75F010A439
:102E7C00FF90024AA3A3E02FF9EA35F0FA90000D77
:102E8C00121F9E900469E0FF782BE68FF0A429F9BD
:102E9C00EA35F0FAEBC0E0EAC0E0E9C0E090024AA3
:102EAC00E0FBA3E0FAA3E0F9900468E075F010A44D
:102EBC00F58285F083121E01FD9004727401F0A35B
:102ECC007404F0A3746CF0D0E0F9D0E0FAD0E0FB1D
:102EDC00122D5D900468E004F0022E59900469E014
:0C2EEC0004F0022E47122D3DE47880F621
:012EF80022B7
:0525540090046CEFF0A3
:10255900E4900472F0A3F090046FF07B019004788A
:1025690004F0A37404F0A37472F01B7A00792E7D31
:10257900161232B012329A900470E0B4120CA3E031
:10258900B4340790046FE04401F0E490046EF090D5
:10259900046EE0C3781E964003022676E490046D2B
:1025A900F090024AE0FBA3E0FAA3E0F990046DE0A1
:1025B900FF75F010A4F58285F083121E01700302E5
:1025C900266D90046CE0606AEF75F010A4FF90022C
:1025D9004AA3A3E02FF9EA35F0FA90000D121F9EE5
:1025E90090046EE0FF782BE68FF0A429F9EA35F024
:1025F900FAEBC0E0EAC0E0E9C0E090024AE0FBA3E0
:10260900E0FAA3E0F990046DE075F010A4F5828575
:10261900F083121E01FD9004787401F0A37404F094
:10262900A37472F0D0E0F9D0E0FAD0E0FB1232B036
:10263900802990024AE0FBA3E0FAA3E0F990046D37
:10264900E075F010A4F58285F083121E01FF900455
:1026590073E02FF0900472E03400F090046DE00410
:10266900F00225AA90046EE004F002259812329A2D
:10267900900470E0B4120CA3E0B4340790046FE046
:082689004402F090046FE0FF31
:012691002226
:100AA70050444343000132000000437261746545BE
:100AB7006E0001009A0132000000436831456E0064
:100AC700000001009D0132000000436832456E00BE
:100AD700000001009E0132000000436833456E00AC
:100AE700000001009F0132000000436834456E009A
:100AF70000000100A00132000000436835456E0088
:100B070000000100A10132000000436836456E0075
:100B170000000100A20132000000436837456E0063
:100B270000000100A30132000000436838456E0051
:100B370000000100A40132000000436839456E003F
:100B470000000100A5013200000043683130456E06
:100B570000000100A6013200000043683131456EF4
:100B670000000100A7013200000043683132456EE2
:100B770000000100A8013200000043683133456ED0
:100B870000000100A9013200000043683134456EBE
:100B970000000100AA013200000043683135456EAC
:100BA70000000100AB0132000000436831364F45B9
:100BB7006E000100AC0132000000526573657400DD
:100BC700000001009B0132000000436C72466C7408
:100BD700000001009C0235000000416C6572740042
:100BE70000000100AF023500000050726573656EAA
:100BF70074000100B10235000000507772476F6F33
:100C070064000100B302350000004F7672546D7026
:100C170000000100B5023500000056494E5F5556E9
:100C270000000100B70235000000494F55545F4FDF
:100C370043000100B90235000000564F55545F4F7D
:100C470056000100BB02350000004F4E4F464600DC
:100C570000000100BD0235000000496E746C6B0096
:100C670000000100C101340000004E54656D7000A2
:100C770000000100C9045A0000015661646A30305F
:100C870000000100CA045A0000015661646A30314D
:100C970000000100CE045A0000015661646A303238
:100CA70000000100D2045A0000015661646A303323
:100CB70000000100D6045A0000015661646A30340E
:100CC70000000100DA045A0000015661646A3035F9
:100CD70000000100DE045A0000015661646A3036E4
:100CE70000000100E2045A0000015661646A3037CF
:100CF70000000100E6045A0000015661646A3038BA
:100D070000000100EA045A0000015661646A3039A4
:100D170000000100EE045A0000015661646A313098
:100D270000000100F2045A0000015661646A313183
:100D370000000100F6045A0000015661646A31326E
:100D470000000100FA045A0000015661646A313359
:100D570000000100FE045A0000015661646A313444
:100D67000000010102045A0000015661646A31352E
:100D7700000001010604180000015664303000002D
:100D8700000001010A041800000156643031000018
:100D9700000001010E041800000156643032000003
:100DA70000000101120418000001566430330000EE
:100DB70000000101160418000001566430340000D9
:100DC700000001011A0418000001566430350000C4
:100DD700000001011E0418000001566430360000AF
:100DE700000001012204180000015664303700009A
:100DF7000000010126041800000156643038000085
:100E0700000001012A04180000015664303900006F
:100E1700000001012E041800000156643130000063
:100E2700000001013204180000015664313100004E
:100E37000000010136041800000156643132000039
:100E4700000001013A041800000156643133000024
:100E5700000001013E04180000015664313400000F
:100E670000000101420418000001566431350000FA
:100E77000000010146041800000156746872303002
:100E8700000001014A0418000001567468723031ED
:100E9700000001014E0418000001567468723032D8
:100EA70000000101520418000001567468723033C3
:100EB70000000101560418000001567468723034AE
:100EC700000001015A041800000156746872303599
:100ED700000001015E041800000156746872303684
:100EE700000001016204180000015674687230376F
:100EF700000001016604180000015674687230385A
:100F0700000001016A041800000156746872303944
:100F1700000001016E041800000156746872313038
:100F27000000010172041800000156746872313123
:100F3700000001017604180000015674687231320E
:100F4700000001017A0418000001567468723133F9
:100F5700000001017E0418000001567468723134E4
:100F670000000101820418000001567468723135CF
:100F770000000101860418000001566D755069785C
:100F8700303001018A0418000001566D75506978E8
:100F9700303101018E0418000001566D75506978D3
:100FA70030320101920418000001566D75506978BE
:100FB70030330101960418000001566D75506978A9
:100FC700303401019A0418000001566D7550697894
:100FD700303501019E0418000001566D755069787F
:100FE70030360101A20418000001566D755069786A
:100FF70030370101A60418000001566D7550697855
:1010070030380101AA0418000001566D755069783F
:1010170030390101AE0418000001566D755069782A
:1010270031300101B20418000001566D755069781E
:1010370031310101B60418000001566D7550697809
:1010470031320101BA0418000001566D75506978F4
:1010570031330101BE0418000001566D75506978DF
:1010670031340101C20418000001566D75506978CA
:1010770031350101C6040600000149303000000087
:1010870000000101CA0406000001493031000000D8
:1010970000000101CE0406000001493032000000C3
:1010A70000000101D20406000001493033000000AE
:1010B70000000101D6040600000149303400000099
:1010C70000000101DA040600000149303500000084
:1010D70000000101DE04060000014930360000006F
:1010E70000000101E204060000014930370000005A
:1010F70000000101E6040600000149303800000045
:1011070000000101EA04060000014930390000002F
:1011170000000101EE040600000149313000000023
:1011270000000101F204060000014931310000000E
:1011370000000101F60406000001493132000000F9
:1011470000000101FA0406000001493133000000E4
:1011570000000101FE0406000001493134000000CF
:1011670000000102020406000001493135000000B9
:1011770000000102060408000009546D70303000B9
:10118700000001020A0408000009546D70303100A4
:10119700000001020E0408000009546D703032008F
:1011A70000000102120408000009546D703033007A
:1011B70000000102160408000009546D7030340065
:1011C700000001021A0408000009546D7030350050
:1011D700000001021E0408000009546D703036003B
:1011E70000000102220408000009546D7030370026
:1011F70000000102260408000009546D7030380011
:10120700000001022A0408000009546D70303900FB
:10121700000001022E0408000009546D70313000EF
:1012270000000102320408000009546D70313100DA
:1012370000000102360408000009546D70313200C5
:10124700000001023A0408000009546D70313300B0
:10125700000001023E0408000009546D703134009B
:1012670000000102420408000009546D7031350086
:1012770000000102460235000000434D4C0000000B
:1012870000000100BF023500000044656275673148
:1012970000000100C3023500000044656275673233
:1012A70000000100C5023500000044656275673320
:1012B70000000100C700000000000000000000005F
:0512C700000000000022
:103C9D00011E0143024AFF0AAC440000000000006F
:103CAD0044000400000000410008004100090042EA
:103CBD00000A000042000C000042000E000042000D
:0D3CCD001000004200120000420014000030
:0527CE0090046CEFF027
:1027D300E4F5A775A4DD75A5B575A6FF12426012D1
:1027E3003E5B12426A7F01123EC9123F34E4FBFD95
:1027F300FF12420DE4FDFF12404FE4FDFF123E23A2
:10280300E4FF1238FF12427A7F01124274E4FB752F
:10281300F004EBA4240AF582E5F03402F583121FD9
:102823006DC479C0000BEBB410E5E4FB75F004EB69
:10283300A424CAF582E5F03400F583121F6D00006D
:10284300000075F004EBA4240AF582E5F03401F5E9
:1028530083121F6D0000000075F004EBA4244AF5F9
:1028630082E5F03401F583121F6D0000000075F05E
:1028730004EBA4248AF582E5F03401F583121F6D7D
:102883000000000075F004EBA424CAF582E5F034DF
:1028930001F583121F6D00000000749D2BF582E487
:1028A3003400F583E4F00BEB64107080E49000C314
:1028B300F0A3F0A3F0A3F0A3F0A3F09000B5F0A36E
:1028C300F090009CF09000BFF0A3F09000BFF0A345
:1028D300F09000B5F0A3F0A3F0A3F0A3F0A3F0A34E
:1028E300F0A3F0A3F0A3F0900098F0A3F0122EF958
:0528F3009000C9EFF0A8
:0128F80022BD
:1041050090FFFF121FF4EFF0850883850982E024F4
:1041150016F582E43400F5837401F0900001021F66
:01412500F4A5
:08000300900462EFF07F00227F
:103C4A00900462EBF0A3EAF0A3E9F0900462E0FBCF
:103C5A00A3E0FAA3E0F9121DE8FF900465E0FBA3D4
:103C6A00E0FAA3E0F9EF121E2E900462E0FBA3E053
:103C7A00FAA3E0F9900001121E01FF900465E0FB2F
:103C8A00A3E0FAA3E0F9900001EF121E407F02229E
:0538FA00900468E0FFEE
:1038FF00EFB41000506790390CF828287302394242
:10390F0002394502394E02395402395A02395D02E1
:10391F00396002396302396602396902395702394F
:10392F005102394B02394802393F02393C7F0B2291
:10393F007F0A227F00227F01227F09227F08227FB8
:10394F0002227F0F227F03227F0E227F04227F0518
:10395F00227F06227F07227F0C227F0D227F0022EB
:1033C400E490046DF0A3F090046CF090046CE0FFC2
:1033D400C3941050171238FF123EC97B077DD37F68
:0C33E4001B12420D90046CE004F080DF2E
:1033F00090046F74E8F00090046FE014F0E070F651
:10340000E490046CF090046CE0FFC39410503A1206
:1034100038FF123EC97DD37F1B12404FEFB4072106
:1034200090046CE0FFC8EFC87E007401088005C3FB
:1034300033CE33CED8F9FF90046DE04EF0A3E04FC9
:10344000F090046CE004F080BC90046DE0FEA3E01A
:01345000FF7C
:013451002258
:1028F900E490046CF0A3F0A3F0A3F0A3F0A3F0FB21
:092909007A027D0B7F101241825D
:10291200900472740AF000900472E014F0E070F611
:0B2922007B207A007D037F10124182B1
:10292D00900472740AF000900472E014F0E070F6F6
:10293D0090046CE0FEA3E04440FF90046CEEF0FECA
:10294D00A3EFF04404FF90046CEEF0A3EFF0A3E0CE
:10295D00FEA3E04480FF90046EEEF0FEA3EFF04482
:10296D0020FF90046EEEF0FAA3EFF0FBCACACBCBBA
:07297D007D0C7F1012418266
:10298400900472740AF000900472E014F0E070F69F
:0F29940090046CE0FAA3E0FB7D0A7F10124182F1
:1029A300900472740AF000900472E014F0E070F680
:0F29B30090046EE0FAA3E0FB7D087F10124182D2
:1029C200900472740AF000900472E014F0E070F661
:1029D200E4FBFA7D097F10124182900470E0FEA3AD
:1029E200E04401FF900470EEF0FEA3EFF04402FF1A
:1029F200900470EEF0A3EFF04408FF900470EEF044
:102A0200A3EFF04410FF900470EEF0FAA3EFF0FB96
:0D2A1200CACACBCB7D047F101241827F0029
:012A1F002294
:10367D0090046C74FFF0E4A3F0A3F07B077DD37F7F
:04368D001B12420DBD
:1036910090046F7464F00090046FE014F0E070F631
:0F36A10090046CE054F7F0FB7D027F1B12420D8A
:1036B00090046F740AF00090046FE014F0E070F66C
:1036C00090046DE04401F04402F04404F0FB7DD22C
:1036D0007F1B12420D7B057DD67F1B12420D7B1096
:1036E0007DD47F1B12420D90046EE04428F0FB7DD8
:1036F000017F1B12420DE4FB7DD57F1B12420D7F23
:0137000000C8
:0137010022A5
:10378600CBEFCBCAEECA7D027F101241827D407F0D
:1037960010123E2390046CEEF0A3EFF0E4FBFA7DEA
:1037A600027F1012418290046CE0540FFEA3E025C4
:1037B600E0FDEE33FCE4121CB5E4FBFA7920784018
:1037C600121B0AE4FBFA79807845121C1390046EEA
:1037D600121F48E4FFFE7D7A7C4490046EE0F8A355
:1037E600E0F9A3E0FAA3E0FB121B0AE4FBFAF9787E
:1037F6003F121A19122C4DE4FBFA797A7844021C0E
:0138060013AE
:0841BC00900014E0FEA3E0FFF7
:1041C400C8EDC8EF088005CEC313CE13D8F97E001E
:0441D4005401FF2271
:103B5500CAEECACBEFCBE0FEA3E0FF900468E0FD20
:103B6500C9EDC9CDEFCDCCEECCC8E9C87E00740156
:103B7500088005C333CE33CED8F9F4FFEEF45CFCF0
:103B8500EF5DFDCEEACECFEBCFCBE9CBC8EBC8EFEF
:103B9500088005C333CE33CED8F9FFEE4CFEEF4D8A
:023BA500FF22FD
:10309100CCEFCCE4900098F0A3F0A3E064016003CE
:1030A1007F0022900098E4F0A304F09000C1E0FEBC
:1030B100A3E0FFCDECCD1241C4EF64014E7002FFDD
:1030C10022900098E4F0A37402F09000AFE0FEA318
:1030D100E0FFCDECCD1241C4EF64014E7002FF223E
:1030E100900098E4F0A37403F09000B5E0FEA3E033
:1030F100FFCDECCD1241C4EF64014E7002FF22906E
:103101000098E4F0A37404F09000B9E0FEA3E0FF9E
:10311100CDECCD1241C4EF64014E7002FF2290004C
:1031210098E4F0A37405F09000BBE0FEA3E0FFCDAE
:10313100ECCD1241C4EF64014E7002FF2290009861
:09314100E4F0A37406F07F012202
:1012CC00E4900469F0A3F0FF123EFF12424CE47B61
:1012DC0064FAF9F8C3121F1F50047F0180027F00CB
:1012EC00900008E070047E0180027E00EF5E7003C7
:1012FC000213BF9000087401F01233C490000AEE80
:0C130C00F0A3EFF09000B1EEF0A3EFF0C2
:1013180090046B740AF00090046BE014F0E070F62F
:06132800E4FFFE1241D8B3
:10132E0090046B7401F00090046BE014F0E070F622
:07133E0074FFFFFE1241D80D
:1013450090046B7464F00090046BE014F0E070F6A8
:10135500E4900468F0900468E0FFC39410505BC803
:10136500EFC890000AE0FEA3E0088005CEC313CEC7
:0C13750013D8F930E03C1238FA123EC9DF
:1013810090046B7464F00090046BE014F0E070F66C
:0313910012367D94
:1013940090046B7464F00090046BE014F0E070F659
:0313A4001228F913
:1013A70090046B7464F00090046BE014F0E070F646
:1013B700900468E004F0809B900027E0700302141B
:1013C70069E4F0FA7B327D05FF12370290009BE05B
:0C13D70064016003021464FFFE1241D8A0
:1013E30090046B7401F00090046BE014F0E070F66D
:1013F30074FFFFFE1241D8E4900468F0900468E0A3
:10140300FFC39410505BC8EFC890000AE0FEA3E04E
:10141300088005CEC313CE13D8F930E03C1238FA56
:03142300123EC9AD
:1014260090046B7464F00090046BE014F0E070F6C6
:0314360012367DEE
:1014390090046B7464F00090046BE014F0E070F6B3
:031449001228F96D
:10144C0090046B7464F00090046BE014F0E070F6A0
:10145C00900468E004F0809BE490009BF0900028DE
:10146C00E06062E4F0FA7B327D05FF1237029000F7
:10147C009CE06401704A900468F0900468E0FFC33B
:10148C009410503CC8EFC890000AE0FEA3E008801E
:10149C0005CEC313CE13D8F930E01D1238FA123E24
:0114AC00C976
:1014AD0090046B7464F00090046BE014F0E070F63F
:1014BD007D037F1B12423E900468E004F080BAE485
:1014CD0090009CF0900008E07003021A1190001635
:1014DD00E0603EE4F090009AE07036900468F09081
:0F14ED000468E0FFC3941050281238FF123EC964
:1014FC0090046B740AF00090046BE014F0E070F64A
:10150C00E4FBFA7D097F10124182900468E004F03C
:10151C0080CEE4900468F0900468E0FFC39410401F
:10152C00030215F4C8EFC890000AE0FEA3E008809F
:10153C0005CEC313CE13D8F920E0030215EB9004AB
:10154C0068E02417F582E43400F583E0700302159B
:10155C00EB900468E0FF2417F582E43400F583E493
:07156C00F01238FF123EC926
:1015730090046B740AF00090046BE014F0E070F6D2
:101583007D797F10123E23900012EEF0A3EFF090CE
:101593000468E0FF249DF582E43400F583E06027CE
:1015A300123091BF0110900013E04420F09000121C
:1015B300E0FAA3E0802A900468E0249DF582E434F5
:1015C30000F583E4F08021900012E0FEA3E0FFE445
:1015D300FBFA7D20123B65900012EEF0A3EFF0E4DE
:1015E300FB7D097F10124182900468E004F002152C
:1015F3002312424CC8ECC8C9EDC9CAEECACBEFCB23
:10160300900000E0FCA3E0FDA3E0FEA3E0240AFFBA
:10161300E43EFEE43DFDE43CFCD3121F1F500302F5
:0D16230016F1900008E0640160030216F16A
:1016300090046B740AF00090046BE014F0E070F614
:10164000E4900468F0900468E0FFC3941040030243
:1016500016E8C8EFC890000AE0FEA3E0088005CEB7
:0F166000C313CE13D8F930E0761238FA123EC910
:10166F0090046B740AF00090046BE014F0E070F6D5
:10167F007D6A7F10123E23900014EEF0A3EFF07DF1
:10168F00061241C49000B3123B559000B3EEF0A385
:10169F00EFF07D021241BC900469EEF0A3EFF0640D
:1016AF00014E702C900468E0FFC8EFC8A3E0FEA3C2
:1016BF00E0088005C333CE33CED8F9FF9000C1E0E8
:1016CF004EF0A3E04FF0E4FBFA7D097F1012418248
:1016DF00900468E004F002164512424C900000128C
:1016EF001F4812424CC8ECC8C9EDC9CAEECACBEFAD
:1016FF00CB900004E0FCA3E0FDA3E0FEA3E0246494
:10170F00FFE43EFEE43DFDE43CFCD3121F1F5003FB
:10171F00021A11900008E064016003021A11FA7BAB
:10172F00327D02FF123702124126900014EEF0A311
:10173F00EFF0E4900468F0900468E0FFC394105059
:10174F001F1238FFCDEFCD1241BC9000AF123B55A9
:10175F009000AFEEF0A3EFF0900468E004F080D7B4
:10176F0090046B740AF00090046BE014F0E070F6D4
:10177F00E4900468F0900468E0FFC3941040030203
:10178F001997C8EFC890000AE0FEA3E0088005CEC5
:10179F00C313CE13D8F920E00302198E1238FA12B0
:0217AF003EC931
:1017B10090046B740AF00090046BE014F0E070F692
:1017C1007D797F10123E23900012EEF0A3EFF0908E
:1017D10000B3E0FEA3E0FF900468E0FD1241C4EF16
:1017E1004E9000136006E06480F08004E04480F0D5
:1017F100900012E0FAA3E0FB7D097F101241827F85
:10180100087E00123786900468E075F004A4248AEB
:10181100F582E5F03401F583121F487F027E001244
:101821003786900468E075F004A4244AF582E5F057
:101831003401F583121F487F017E00123786900420
:1018410068E075F004A4240AF582E5F03401F5831B
:10185100121F487F107E00123786E4FBFA79A078C8
:1018610041121B0A7B6F7A127903783B121C139089
:101871000468E075F004A424CAF582E5F03401F5AA
:0418810083121F4867
:1018850090046B740AF00090046BE014F0E070F6BD
:101895007D797F1B123E23900014EEF0A3EFF07DBF
:1018A500091241C4CAEECACBEFCB9000BF123B5B15
:1018B5009000BFEEF0A3EFF07D0A1241BCCAEECA5C
:1018C500CBEFCB9000B5123B5B9000B5EEF0A3EFEC
:1018D500F0900014E0FEA3E0FF7D0B1241C4CAEEB8
:1018E500CACBEFCB9000B7123B5B9000B7EEF0A3ED
:1018F500EFF0900014E0FEA3E0FF7D0C1241C4CA96
:10190500EECACBEFCB9000B9123B5B9000B9EEF07D
:10191500A3EFF0900014E0FEA3E0FF7D0D1241C49B
:10192500CAEECACBEFCB9000BB123B5B9000BBEE7F
:10193500F0A3EFF0900014E0FEA3E0FF7D0E12414E
:10194500C4CAEECACBEFCB9000BD123B5B9000BD85
:10195500EEF0A3EFF0900468E0B4012D900014E0E0
:10196500FFA3E090000CCFF0A3EFF0900098E0FF0C
:10197500A3E090000ECFF0A3EFF07D797F10123E2B
:1019850023900010EEF0A3EFF0900468E004F0025D
:101995001784900009E070047F0180027F009000A9
:1019A50009EFF0E4900468F09000C9E0FE90046847
:1019B500E0FFC39E50201223DE900468E075F0041A
:1019C500A4240AF582E5F03402F583121F48900439
:1019D50068E004F080D212424C900004121F489037
:1019E500000CE0FFA3E09000C3CFF0A3EFF0900060
:1019F5000EE0FFA3E09000C5CFF0A3EFF09000103C
:0C1A0500E0FFA3E09000C7CFF0A3EFF0DB
:011A110022B2
:103E5B00E4F5A7D2927B087D0AFF123FCAE4FBFD73
:103E6B00FF123FCAE4FB7D01FF123FCA7B087D0AAC
:103E7B007F01123FCA7BFFE4FD7F01123FCA7BFF2C
:073E8B007D017F01023FCA27
:103FCA0090046EEFF0A3EDF0A3EBF01242809004A0
:103FDA006EE0540725E04440FF12409C90046FE0D5
:0F3FEA00FF12409C900470E0FF12409C02428640
:1041D80090046CEEF0A3EFF0FB7D14E4FF123FCAED
:0C41E80090046CE0FB7D15E4FF023FCA70
:083F680090046CEFF0A3EDF0F2
:103F700012428090046CE0540725E04441FF124057
:103F80009C90046DE0FF12409C12414590046EEF3E
:093F9000F012428690046EE0FF7D
:013F99002205
:104126007D137F01123F68EF7F00FEC007C0067D4A
:0E413600120F123F68EFFDD0E0FED0E04DFF0B
:014144002258
:0A426000E4F5A7C280C282D28322D7
:06428000E4F5A7C2832251
:06428600E4F5A7D283223B
:10409C00E4F5A7FEEF5480D394004003D38001C312
:1040AC009282EF25E0FFD280D280D280C2800EEEC9
:0540BC00B408E1C2821E
:0140C10022DC
:10414500E4F5A7FFC282FEEF25E0FFA281E4334F2D
:0E415500FFD280D280D280C2800EEEB408E984
:014163002239
:0A426A00E4F5A7D2A1D286D2872284
:073FF900E4F5A7D286D28790
:104000009004737406F000900473E014F0E070F60E
:02401000C28666
:104012009004737406F000900473E014F0E070F6FC
:03402200C2872230
:043E9200C286D2878B
:103E96009004737406F000900473E014F0E070F67A
:023EA600D286C2
:103EA8009004737406F000900473E014F0E070F668
:103EB8009004737406F000900473E014F0E070F658
:013EC80022D7
:04345200EF25E0FF83
:10345600E4FEEF5480D394004003D38001C39286E8
:04346600EF25E0FF6F
:10346A009004747406F000900474E014F0E070F6AE
:02347A00D287F7
:10347C009004747406F000900474E014F0E070F69C
:02348C00C287F5
:10348E009004747406F000900474E014F0E070F68A
:07349E000EEEB408B5D28662
:1034A5009004747406F000900474E014F0E070F673
:0234B500D287BC
:1034B7009004747406F000900474E014F0E070F661
:0A34C700A286E433900473F0C2877C
:0E34D100A37406F000900474E014F0E070F6AE
:0134DF0022CA
:02333000D28643
:103332009004727406F000900472E014F0E070F6EB
:03334200E4FEFDA9
:103345009004727406F000900472E014F0E070F6D8
:02335500D2871D
:103357009004727406F000900472E014F0E070F6C6
:0C336700EE25E0FEA286E4334EFEC28795
:103373009004727406F000900472E014F0E070F6AA
:0A3383000DEDB408BDEF24FF9286A3
:10338D009004727406F000900472E014F0E070F690
:02339D00D287D5
:10339F009004727406F000900472E014F0E070F67E
:0233AF00C287D3
:1033B1009004727406F000900472E014F0E070F66C
:0233C100AF0655
:0133C30022E7
:103F3400123FF97FE11234567F01123330AB07127E
:103F44003E92123FF97FE31234567F01123330124E
:103F54003E92EB30E3055407FC8006EF5407240837
:033F6400FCAF04AB
:013F67002237
:103EC900EFC394085008EF4408FCE4FD8008E4FCC3
:103ED900EF24F84408FD123FF97FE0123456AF048D
:103EE900123456123E92123FF97FE2123456AF0550
:063EF900123456023E9255
:10420D00123FF9123452AF05123456AF0312345621
:03421D00023E92CC
:0E423E00123FF9123452AF05123456023E926E
:02404F00AC07BC
:10405100123FF9EC25E0FF123456AF051234561227
:104061003FF9AF04EF25E04401FF1234567F0112FE
:054071003330023E9215
:02418200AC0788
:10418400EAF9123FF9AF04123452AF05123456AFB4
:0C41940001123456AF03123456023E9262
:023E2300AC07EA
:103E2500123FF9EC25E0FF123456AF051234561255
:103E35003E92123FF9AF04EF25E04401FF123456DC
:103E4500E4FF123330AC077F01123330AD07123E69
:053E550092ECFEEDFF00
:013E5A002245
:0B3CDA004103910044038D0000000036
:0F3D6B00C295C2947FF47E01123881D294D29512
:103D7A0090047B744BF00090047BE014F0E070F642
:0B3D8A007E002096047F0180027F0075
:103D950090047B74F4F00090047BE014F0E070F67E
:043DA500D294C2955D
:013DA90022F7
:093BA700D294C295C294EF6012A1
:103BB00090047B740FF00090047BE014F0E070F64A
:023BC000801073
:103BC20090047B7469F00090047BE014F0E070F6DE
:053BD200D294EF601128
:103BD70090047B7469F00090047BE014F0E070F6C9
:013BE70022BB
:103BE80090047B740FF00090047BE014F0E070F612
:013BF80022AA
:023DE900A90728
:103DEB00E4FDFCAF057E007401A807088005C33312
:103DFB00CE33CED8F9FFE9FBEF5BD39400748094FC
:103E0B008040047F0180027F00123BA70DBD0001A3
:073E1B000CED64084C70CCB3
:013E2200227D
:063DAA00D294C295C29400
:103DB00090047B740AF00090047BE014F0E070F64D
:023DC000D2959A
:103DC20090047B7414F00090047BE014F0E070F631
:063DD200A296E4FE33FF9F
:103DD80090047B7450F00090047BE014F0E070F6DF
:013DE80022B8
:05429600D294C2952244
:10402500E4FDFC123DAAEF4E60137E007401A80466
:10403500088005C333CE33CED8F9FF80027F00EF69
:094045004DFD0CECB408DCAF05E4
:01404E00224F
:102EF900123D6B7FCC123DE97F99123DE97F5A1251
:102F09003DE97FA5123DE912429612402590046DD4
:102F1900E4F0A3EFF07FF47E01123881E49003918D
:102F2900F07F00123EFF123D6B7F0F123DE9E4FB7B
:102F3900FA124025900391E075F008A424D2F58295
:102F4900E43403F583E5822BF582E5833AF583EFD3
:102F5900F00BBB00010AEB64084A70D5900391E0BD
:102F690075F008A424D2F582E43403F583E0F46013
:102F7900267F99123DE97F96123DE97F69123DE965
:102F890012402590046DE4F0A3EFF0900391E00462
:102F9900F0E0C39410408A7F0A7E00123D2C123D56
:102FA9006B7FCC123DE97F99123DE97F3C123DE9E7
:102FB9007FC3123DE912429612402590046DE4F058
:082FC900A3EFF0900391E0FF7B
:012FD10022DD
:0523DE0090046CEFF01B
:1023E30012424CA804A905AA06AB0790038DE0FC92
:1023F300A3E0FDA3E0FEA3E0244BFFE43EFEE43DA7
:10240300FDE43CFCD3121F1F5003022537E4900464
:102413006FF0A3F0900391E0FFC3900470E09F740A
:1024230080F890046FE0648098400302251E7F00CB
:10243300123EFF123D6BEF4E7018FE7F807DFF7BD7
:10244300017A0379D2122025E4900391F0FFFEFD77
:10245300FC227F55123DE9E490046DF0A3F0900453
:102463006DE0FCA3E0FDC39408EC648094805036D7
:10247300A3E0FEA3E07803C333CE33CED8F924D24E
:10248300F58274033EF583E5822DF582E5833CF501
:1024930083E0FF123DE990046EE004F070C0900405
:1024A3006DE004F080B87FBE123DE9124025900430
:1024B30071EFF0124025900472EFF0FE900471E08A
:1024C300FDEEFCEC121CB5E4FBFA79AA7842121B70
:1024D3000AE4FBFA79AA7844121C13C004C005C0AD
:1024E30006C00790046FE0FEA3E07802C333CE3347
:1024F300CED8F92492F58274033EF583D007D00633
:10250300D005D004121F48900470E004F060030269
:10251300241790046FE004F0022417123D6B7FCC64
:10252300123DE97F44123DE912429612424C900358
:102533008D121F4890046CE025E025E02492F5827B
:10254300E43403F583E0FCA3E0FDA3E0FEA3E0FF96
:012553002265
:101A1200021D23E86480F8E933E83360110460F0C2
:101A2200ED33EC337009E8FCE9FDEAFEEBFF22043A
:101A320060DED3EB9FEA9EE99DE8C2E78CF0C2F735
:101A420095F0400CE8CCF8E9CDF9EACEFAEBCFFB01
:101A5200121CEE85D0F05804700320D5B3E8047050
:101A6200075002B2D5021D2D92D5EC0460F7E4CCEA
:101A7200C0E0C398F8603B94186008400DD0E0FBCA
:101A8200021D05E4FBFAC9FC8028E830E406E4C93B
:101A9200FBE4CAFCE830E305E4C9CACBFCE854071E
:101AA2006010F8C3E913F9EA13FAEB13FBEC13FC29
:101AB200D8F130F52FC3E49CFCEF9BFFEE9AFEEDCC
:101AC20099FDD0E0FBEF4E4D4C701222DB03021D5C
:101AD2002AEC2CFCEF33FFEE33FEED33FDED30E765
:101AE200EB021D05EF2BFFEE3AFEED39FDD0E0FBD8
:101AF20050130BBB0003021D2DED13FDEE13FEEF81
:081B020013FFEC13FC021D05AA
:101B0A00EC4D6011E8497017ED33EC3304600DE4D5
:101B1A00FCFFFEFD22E933E8330470F8021D2312AC
:101B2A001CEE58046009E4CC2481500628500902AE
:101B3A001D2D284003021D2AC0E0EB4A7044B980DB
:101B4A0006D0E0FB021D19EF4E701CBD8008EBFFAA
:101B5A00EAFEE9FD80EBE98DF0A4FEE5F0021BF355
:101B6A00E9CDF9EAFEEBFFEF89F0A4FCE5F0CE89B6
:101B7A00F0A42EFFE435F0CD89F0A42DFEE435F073
:101B8A008067EF4E7005BD80D780C3EF8BF0A4ACA1
:101B9A00F0EE8BF0A42CFCE435F0F8EF8AF0A42CDC
:101BAA00E5F038FCE433CB8DF0A42CFCE5F03BF8EF
:101BBA00EE8AF0A42CFCE5F038F8E433CF89F0A4DF
:101BCA002CFCE5F038CF3400CE89F0A42FFFE5F0E5
:101BDA003EFEE433C98DF0A42EFEE5F039CD8AF03D
:101BEA00A42FFFE5F03EFEE43DFD33D0E0FB5007B5
:101BFA000BBB000F021D2DEC2CFCEF33FFEE33FE66
:061C0A00ED33FD021D0593
:101C1000021D2DEC5D046005E859047003021D23CC
:101C2000121CEE580460F6EC4860F2EC7004FDFE05
:101C3000FF22C860DB2481C85009C39860025006A7
:101C4000021D2A9850CAF582E9294B4A7005AB82D9
:101C5000021D1975F0007C1A7880C3EF9BEE9AED97
:101C600099400DC3EF9BFFEE9AFEED99FDE842F01F
:101C7000DC23ACF0D0E0FFD0E0FED0E0FDAB822072
:101C8000E7101BEB60BAEC2CFCEF33FFEE33FEEDFC
:101C900033FD021D05E803F830E705C0F075F000DC
:101CA000EF2FFFEE33FEED33FD40B830E7C280AAE0
:101CB00075F020800E75F010800575F0087D007EAF
:101CC000007F003392D530D503121F11EC33401042
:101CD000EF33FFEE33FEED33FDEC33FCD5F0ED22B8
:0E1CE000E5F0247EA2D513CC92E7CDCEFF22F4
:102C4D00900472121F4874FFFFFEFDFC900472E0A9
:102C5D00F8A3E0F9A3E0FAA3E0FBC3121F1F60384D
:102C6D007F807E967D187C4B900472E0F8A3E0F98E
:102C7D00A3E0FAA3E0FB121D386002501B7F807E9B
:102C8D00967D187CCB900472E0F8A3E0F9A3E0FAEE
:102C9D00A3E0FB121D38500F900472E0FCA3E0FD81
:102CAD00A3E0FEA3E0FF22900472E0FCA3E0FDA3ED
:102CBD00E0FEA3E0FF121DB1900476121F489004B0
:102CCD0076E0FCA3E0FDA3E0FEA3E0FFEC121CB058
:102CDD00C8ECC8C9EDC9CAEECACBEFCB900472E0FF
:102CED00FCA3E0FDA3E0FEA3E0FF121A15E4FBFA3E
:102CFD00F9F8121D3860264024900476E0FCA3E01C
:102D0D00FDA3E0FEA3E0FFEF24FFFFEE34FFFEED99
:102D1D0034FFFDEC34FFFC900476121F48900476CE
:102D2D00E0FCA3E0FDA3E0FEA3E0FFEC121CB0224B
:101CEE00E9D2E7C933E833F892D5EDD2E7CD33EC3C
:071CFE0033FC5002B2D522B5
:101D0500EC30E7100FBF000C0EBE00080DBD00043F
:101D15000BEB6014A2D5EB13FCED92E7FD2274FFEB
:101D2500FCFDFEFF22E480F8A2D574FF13FC7D8044
:031D3500E480EF58
:101D380074F8CC6480CCC86480C8F58204604FC352
:101D4800EB9FF5F0EA9E42F0E99D42F0E89C45F0F1
:101D5800603C501DE5825FFFE582D313CB5BCBF47B
:101D68002B5582FB50280ABA002409B900200880A4
:101D78001DE5825BFBE582D313CF5FCFF4C3132F3E
:101D88005582FF50090EBE00050DBD00010CC3EBC6
:101D98009FF5F0EA9E42F0E99D42F0E89C45F0602C
:091DA80007CC4820E701B3EC224E
:101DB100EDD2E7CD33EC3392D524814006E4FFFE2A
:101DC100FDFC22FCE4CFCECDCC24E0501174FF8089
:101DD100EDC3CC13CCCD13CDCE13CECF13CF047026
:071DE100F030D5DE021F11F6
:030000000234E0E7
:0C34E000787FE4F6D8FD75818102352765
:101DE800BB010689828A83E0225002E722BBFE02F9
:091DF800E32289828A83E493222C
:101E0100BB010CE58229F582E5833AF583E0225096
:101E110006E92582F8E622BBFE06E92582F8E222E0
:0D1E2100E58229F582E5833AF583E49322FA
:101E2E00BB010689828A83F0225002F722BBFE0193
:021E3E00F3228D
:101E4000F8BB010DE58229F582E5833AF583E8F0D8
:101E5000225006E92582C8F622BBFE05E92582C884
:021E6000F2226C
:101E6200C2D5EC30E709B2D5E4C39DFDE49CFCEE9B
:101E720030E715B2D5E4C39FFFE49EFE122051C3A2
:101E8200E49DFDE49CFC800312205130D507C3E49D
:061E92009FFFE49EFE220A
:101E9800C5F0F8A3E028F0C5F0F8E58215827002D5
:061EA8001583E038F02272
:101EAE00BB010A89828A83E0F5F0A3E022500687FF
:101EBE00F009E71922BBFE07E3F5F009E3192289C1
:0B1ECE00828A83E493F5F074019322F4
:101ED900BB010789828A83021E98500B09C5F02726
:101EE900F7C5F01937F722BBFE0D09F8E325F0F322
:101EF900C5F019E338F322F889828A83740193259E
:081F0900F0C5F0F8E493382262
:0E1F1100C3E49FFFE49EFEE49DFDE49CFC22E1
:101F1F00EB9FF5F0EA9E42F0E99D42F0E89C45F018
:011F2F00228F
:0C1F3000E6FC08E6FD08E6FE08E6FF22DD
:0C1F3C00ECF608EDF608EEF608EFF622D1
:0C1F4800ECF0A3EDF0A3EEF0A3EFF0220C
:101F5400D083D082E493F608740193F60874029354
:091F6400F608740393F67404738B
:101F6D00A8828583F0D083D082121F84121F841221
:101F7D001F84121F84E473E493A3C583C5F0C58346
:101F8D00C8C582C8F0A3C583C5F0C583C8C582C8BE
:011F9D002221
:101F9E00BB010DE58229F582E5833AF5830220C562
:101FAE005007E92582F80220BCBBFE07E92582F81E
:101FBE000220CEE58229F582E5833AF5830220D709
:101FCE00D083D082F8E4937012740193700DA3A3A2
:101FDE0093F8740193F5828883E4737402936860B6
:061FEE00EFA3A3A380DFB6
:101FF400E5092582F582E5083583F583B50804856E
:1020040082092210AF06858209F50822858209F526
:0420140008D2AF221D
:0D201800E5092582F582E5083583F5832270
:1039DD0090046CEBF0A3EAF0A3E9F0E4900474F02A
:1039ED00A3F090047274FFF5F01220A645F0603C30
:1039FD0090046FE0FBA3E0FAA3E0F9121DE8FF903D
:103A0D00046CE0FBA3E0FAA3E0F9900474E475F014
:103A1D00011220A685F082F583EF121E40EF60C2E1
:103A2D00900470E475F001121E9880B690046CE05D
:083A3D00FBA3E0FAA3E0F9226B
:1038070090046FEBF0A3EAF0A3E9F0A3EBF0A3EACF
:10381700F0A3E9F0900472E0FBA3E0FAA3E0F91249
:103827001DE8600C900473E475F001121E9880E4A3
:10383700900472E0FBA3E0FAA3E0F9121DE86D70B3
:10384700012290046FE0FBA3E0FAA3E0F9EBC0E0EC
:10385700EAC0E0E9C0E0A3E0FBA374FFF5F01220A3
:10386700A6FAD082D083D0E06B7009E5F06582704C
:0A38770003EA658370BAFBFAF92238
:10202500EF4E6012EF60010EEDBB010B89828A83D2
:10203500F0A3DFFCDEFA2289F05007F709DFFCA9DF
:0C204500F022BBFEFCF309DFFCA9F02236
:1034EC00024164E493A3F8E493A34003F68001F251
:1034FC0008DFF48029E493A3F85407240CC8C333E1
:10350C00C4540F4420C8834004F456800146F6DFAF
:10351C00E4800B0102040810204080903C9AE47E69
:10352C00019360BCA3FF543F30E509541FFEE493A4
:10353C00A360010ECF54C025E060A840B8E493A36B
:10354C00FAE493A3F8E493A3C8C582C8CAC583CA96
:10355C00F0A3C8C582C8CAC583CADFE9DEE780BE4E
:013CE50000DE
:10205100BC000BBE0029EF8DF084FFADF022E4CC73
:10206100F875F008EF2FFFEE33FEEC33FCEE9DEC3C
:10207100984005FCEE9DFE0FD5F0E9E4CEFD22ED82
:10208100F8F5F0EE8420D21CFEADF075F008EF2FCC
:10209100FFED33FD4007985006D5F0F222C398FDBD
:0520A1000FD5F0EA225A
:1020A600A3F8E0C5F025F0F0E582158270021583ED
:0620B600E0C838F0E8224A
:0920BC00E6FB08E6FA08E6F92249
:0920C500E0FBA3E0FAA3E0F9221C
:0920CE00E2FB08E2FA08E2F92243
:0C20D700E493FB740193FA740293F92265
:00000001FF
